:020000040000FA
:04000000D7EF24F022
:08000800056ED8CF06F0E0CF31
:1000100007F00001E9CF0DF0EACF08F0E1CF09F0D9
:10002000E2CF0AF0D9CF0BF0DACF0CF0F3CF14F017
:10003000F4CF15F0FACF16F000C00FF001C010F0A9
:1000400002C011F003C012F004C013F09DA22CEF07
:1000500000F09EB26EEF01F09DA032EF00F09EB076
:10006000E4EF01F00FC000F010C001F011C002F089
:1000700012C003F013C004F00E8E0DC0E9FF08C0DB
:10008000EAFF09C0E1FF0AC0E2FF0BC0D9FF0CC0C4
:10009000DAFF14C0F3FF15C0F4FF16C0FAFF0550D5
:1000A00007C0E0FF06C0D8FF1000F2CF0EF0F29EAE
:1000B000F76AC40FF66E000EF7220900F5500EBE67
:1000C000F28E12000000320062008E00B500D500F2
:1000D000ED00FB000001FB00ED00D500B5008E0037
:1000E000620032000000CEFF9EFF72FF4BFF2BFF2D
:1000F00013FF05FF00FF05FF13FF2BFF4BFF72FFF0
:100100009EFFCEFFF2CF0EF0F29EF76A1E0FF66E44
:10011000010EF7220900F5500EBEF28E120000808B
:1001200040C020A060E0109050D030B070F008883F
:1001300048C828A868E8189858D838B878F80484C7
:1001400044C424A464E4149454D434B474F40C8CDF
:100150004CCC2CAC6CEC1C9C5CDC3CBC7CFC028273
:1001600042C222A262E2129252D232B272F20A8ADF
:100170004ACA2AAA6AEA1A9A5ADA3ABA7AFA068667
:1001800046C626A666E6169656D636B676F60E8E7F
:100190004ECE2EAE6EEE1E9E5EDE3EBE7EFE018119
:1001A00041C121A161E1119151D131B171F10989AF
:1001B00049C929A969E9199959D939B979F9058537
:1001C00045C525A565E5159555D535B575F50D8D4F
:1001D0004DCD2DAD6DED1D9D5DDD3DBD7DFD0383E3
:1001E00043C323A363E3139353D333B373F30B8B4F
:1001F0004BCB2BAB6BEB1B9B5BDB3BBB7BFB0787D7
:1002000047C727A767E7179757D737B777F70F8FEE
:100210004FCF2FAF6FEF1F9F5FDF3FBF7FFFF2CF4B
:100220000EF0F29EF76A380FF66E020EF722090002
:10023000F5500EBEF28E12002530344C583030305E
:1002400038000201CA6BCB6B92948994C950610E3D
:10025000C96EC730FEE3C950C96AC730FEE3C95052
:10026000036ACA6F03C0CBF2CAC203F0000ECA6FA2
:1002700003C0CBF2C950C96AC730FEE3C950CA13E4
:10028000CB31036ECA31026E033202323F0E0316C7
:1002900002C0CAF203C0CBF2000B006ECB51200BA0
:1002A000036E0050031002E0C00ECB1392948984B9
:1002B000CAC201F0CBC202F00001000C92948994F2
:1002C0000201C9518009CA11CC6FC950CCC2C9FF03
:1002D000C730FEE3929489840001000C01012F2DA8
:1002E0006FD0D8902935026E2A35036E0250390F2F
:1002F000016E000E032201C0C8F203C0C9F2000162
:10030000A0DF01C0CAF201013051080DF350020113
:10031000CD6BCC6F036A01013051460FE96E010EBF
:100320000320EA6ED890EF34036A0201CC25016EF7
:10033000CD51032201504E0FE96E010E0320EA6EEB
:10034000ECCF03F0ED52EF50CA5D006E035002583F
:10035000C9C2EAFFC8C2E9FFEC6EED5200C0EFFF70
:100360000101302B3051030801E2306B036A305138
:10037000320FE96E010E0320EA6EEFCFC8F230C1F2
:10038000C9F2C8C2CAF2000199DF0101292BD8B411
:100390002A2B29513C0808E12A5306E12E6B2D6BCC
:1003A0002C6B010E2B6F0CD02951780809E12A53D0
:1003B00007E12E6B2D6B2C6B020E2B6F2A6B296BBA
:1003C0009E92000132EF00F0FB0ECF6E1D0ECE6E3E
:1003D0000201C86BC851030817E3C851080DF35058
:1003E000CA6BC96F040EC925016E000ECA21036EC7
:1003F0000150190FE96E000E0320EA6E010EEE2681
:1004000001E3EF2AC82BE6D79E90000132EF00F0FF
:1004100002015D6B5D5103081DE35E6B5E510308D5
:1004200017E35D51080DF350606B5F6FD8905E3538
:10043000036A5F25016E6051032201504E0FE96E81
:10044000010E0320EA6EEC6AED52EF6A5E2BE6D7EE
:100450005D2BE0D7000181EF15F0020EEA6EB10EC0
:10046000E96EEF500EE00C0E016E006A002EFED712
:10047000012EFBD7F70E006E002EFED700D0EF2E18
:10048000F2D7000C51C2D7FF50C2D6FF02016CC296
:10049000E9FF6DC2EAFFEC6AED52EF6A020E6C25CD
:1004A000E96E000E6D21EA6EEF6A030E6C25E96EAF
:1004B000000E6D21EA6EEF6A040E6C25E96E000EE7
:1004C0006D21EA6EEF6A050E6C25E96E000E6D2156
:1004D000EA6EEF6A0001000C92948994C950180EDC
:1004E000C96EC730FEE3C950C96AC730FEE39294B3
:1004F000898490EF02F09294899402015EC260F2C6
:10050000C9505EC2C9FFC730FEE3C9505FC2C9FF10
:10051000C730FEE392948984000197EF02F0DCD7A4
:10052000070E02015E6F3E0E5F6F0001E4D7969EDC
:100530008D9E968C02015D6B84BC5D2B0001BBEF30
:1005400015F0010E0201795D006E000E7A59016E00
:10055000000E7B59026E000E7C59036E846B836B18
:10056000826B010E816F0050856F07E0D890813754
:10057000823783378437852FF9D7806B7F6B7E6B0B
:100580007D6B80517C5D43E30BE17F517B5D3FE3FD
:1005900007E17E517A5D3BE303E179517D5D37E20E
:1005A00094908B80030E006E002EFED7815175153E
:1005B000006E82517615016E83517715026E84515B
:1005C0007815036E005206E1015204E1025202E185
:1005D000035203E094928B8202D094928B92030E8A
:1005E000006E002EFED794908B90030E006E002EAE
:1005F000FED7D8908433833382338133010E7D2735
:10060000D8B07E2BD8B47F2BD8B4802BBAD70001BA
:10061000000C0201786B776B766B72C275F27C6BA3
:100620007B6B7A6B080E796F00018BDF0201786BB0
:10063000776B74C276F273C275F27C6B7B6B7A6BEC
:10064000100E796F00017DDF3BEF03F0D8900201BF
:100650006E35716F718994908B9092968996210E68
:10066000006E002EFED771C272F270C274F26FC2B9
:1006700073F20001CED7210E006E002EFED79296A7
:10068000898694928B9294908B90000C02016E6BF1
:10069000706B6F6B0001DADF010E02016E6F706B21
:1006A0006F6B0001D3DF020E02016E6F706B6F6B18
:1006B0000001CCDF030E02016E6F706B6F6B0001E7
:1006C000C5DFBDEF15F08E0E006EADC201F0ACC2FD
:1006D00002F0036A01AE05D0011E021E022A01E1EA
:1006E000012A015209E102C001F0026A080E005E0F
:1006F000015202E1006A0DD0D89001BE04D002364A
:1007000001360006F9D70201ADAF02D0000101D0D9
:10071000019E0001000CABC2B2F20201AF51B21B4C
:10072000B2AF05D0D894D890ABBFD8802FD0ABC291
:10073000B2F2AEC2B3F2AA51B35F06E0B2AF26D0B6
:10074000D850010AD86E22D0AFC2B3F2AB51B35F1A
:1007500006E0B2AF1BD0D850010AD86E17D0B0C295
:10076000B3F2AC51B35F06E0B2AF10D0D850010A7B
:10077000D86E0CD0B1C2B3F2AD51B35F06E0B2AFE8
:1007800005D0D850010AD86E01D0D8900001000CD5
:10079000800ED8A202D00201B31B0201B86BB96B64
:1007A000AFC2B7F2B351B71BAE51D8B4DFD0B66FFA
:1007B000006EB251D8B4E3D0B65FD8B483D03EE374
:1007C000B3C2BCF2BC8FB4C2BBF2B5C2BAF2B96B51
:1007D000D890BC33BB33BA33B933B62FF8D7B7AFE1
:1007E00003D0B881E0D0B891B691B889020EEA6E14
:1007F000B10EE96EEBD0B899B7BF0AD0B6A113D04D
:10080000BC33BB33BA33B933002AD8B4C7D00BD00A
:10081000BCBF0CD0D890B937BA37BB37BC3700064D
:10082000D8B4BCD0F5D7B88D6DD0B89DAFC2B7F2F3
:10083000AFAF02D0BC8FABD0BC9FA9D0B2C2B6F2D2
:10084000B2C200F0AE51B65FAFC2BCF2BC8FB0C254
:10085000BBF2B1C2BAF2B96BD890BC33BB33BA3376
:10086000B933B62FF8D7B7AF03D0B8839CD0B893BD
:10087000B691B88B020EEA6EB50EE96EA7D0B89BA2
:10088000B7BF0AD0B6A113D0BC33BB33BA33B93328
:10089000002AD8B483D00BD0BCBF0CD0D890B937C5
:1008A000BA37BB37BC370006D8B478D0F5D7B88F85
:1008B00029D0B89FB3C2B7F2B3AF02D0BC8F67D014
:1008C000BC9F65D0B3C2BCF2BC8FB4C2BBF2B5C290
:1008D000BAF2B7AF04D0BC9FB88565D0B895B96BF4
:1008E000B691020EEA6EB10EE96E70D0B7BF1CD0A1
:1008F000AFC2B7F2B6A106D0BC33BB33BA33B933FB
:10090000002A4CE0B9AF0BD0BA2B09E1BB2B07E1B1
:10091000BC2B05E1BC33BB33BA33002A3FE0B8BD82
:1009200084D7B8BFC6D71CD0800EBC1BBCAF04D0C8
:100930003AD0B3C2B7F20AD0AFC2B7F2BC5306E1A5
:10094000BB5304E1BA5302E1006A21D0BCBF08D016
:10095000D890B937BA37BB37BC37002EF7D71ED07F
:10096000B7AF02D0BC8F13D0BC9F11D0B2C200F081
:10097000B3C2BCF2B4C2BBF2B5C2BAF208D0AEC2C6
:1009800000F0AFC2BCF2B0C2BBF2B1C2BAF2BCC29C
:1009900001F0BBC202F0BAC203F034D0006A016AAF
:1009A000026A036A2FD0B96BBA1FBB1FBC1FB91FE5
:1009B000B92B05E1BA2B03E1BB2B01E1BC2BB8B18C
:1009C00012D7B8B354D7B8B589D7B3D7EF50BA2731
:1009D00005E3BB2B03E1BC2BD8B4B681ED52EF503D
:1009E000BB2703E3BC2BD8B4B681ED52EF50EFBE6A
:1009F00001D0800ABC27D8B0B681B8B9FCD6B8BB44
:100A00003ED774D70001000C0201AE51D8B4A5D076
:100A1000BA6FB251D8B4A1D0BA5F05E37F0EBA273E
:100A2000D8B09BD006D0810EBA5FD8A096D0D8B4EB
:100A300094D0BAC200F0016A026A036AB96BAFC20D
:100A4000B8F2B88FB0C2B7F2B1C2B6F2190EBA6F2F
:100A5000B551B65F0DE2010EB75F0AE2B85F08E27A
:100A6000B95F06E2B92BB82BB72BB551B62728D002
:100A7000B451B75F12E2010EB85F0FE2B95F0DE249
:100A8000B92BB82BB451B727B551B62719E3B72BFB
:100A900017E1B82B15E1B92B13D0B3518009B85F1A
:100AA0000EE2010EB95F0BE2B92BB3518009B827F2
:100AB000B451B727E9E3B82BE7E1B92BE5D70380B9
:100AC000BA2F01D00BD0D890B637B737B837B9376F
:100AD000D890033602360136BB37BAD7BBA106D051
:100AE000D890013202320332BB3302D0000635E027
:100AF000BBBF1ED0D890B637B737B837B937B55166
:100B0000B65F07E2010EB75F04E2B85F02E2B95FC9
:100B10001AE3B451B75F05E2010EB85F02E2B95FB4
:100B200012E3B3518009B85F03E2010EB95F0BE332
:100B3000032A09E1022A07E1012A05E1002A0DE062
:100B4000013202320332AFC2BAF2B351BA1BBAAFAA
:100B500002D0018E06D0019E04D0006A016A026AAA
:100B6000036A0001000C0201AA51D8B471D0006ED2
:100B7000AE51D8B46DD0002604E3810E002668E2A1
:100B800004D07F0E005E64E363E0ABC2B2F2AF510B
:100B9000B21BAB8FAF8FAD51B103F4CFB4F2AC51F8
:100BA000B003F4CF03F0F3CFB3F2B103F350B427A3
:100BB000F450B323000E0322AD51B003F350B42719
:100BC000F450B323000E026A03220222AB51B10398
:100BD000F350B327F4500322000E0222AB51B003AE
:100BE000F3500326F4500222000E016A0122AD5197
:100BF000AF03F350B327F4500322000E0222012268
:100C0000AC51AF03F3500326F4500222000E012230
:100C1000AB51AF03F3500226F4500122002A01BE6B
:100C200005D0B3370336023601360006000EB3AFE7
:100C30000AD0032A02220122015005E1025003E1F9
:100C4000035001E1002AB2BF018EB2AF019E04D071
:100C5000006A016A026A036A0001000C98C29CF2F1
:100C600097C29BF296C29AF295C299F29CC2ADF2DB
:100C70009BC2ACF29AC2ABF299C2AAF20201B16B6A
:100C8000B06BAF6B7F0EAE6F000145DDD8B436D2CE
:100C9000020E0201AB6F990EE96EABC2EAFF7E0E47
:100CA000EF6ED8829CC2B1F29BC2B0F29AC2AFF290
:100CB00099C2AEF2B56BB46BB36B7F0EB26F00012D
:100CC00067DD00C0AAF201C0ABF202C0ACF203C003
:100CD000ADF2D8929CC2B1F29BC2B0F29AC2AFF20E
:100CE00099C2AEF20201B56BB46BB36B7F0EB26FFB
:100CF00000014EDDADC2B1F2ACC2B0F2ABC2AFF298
:100D0000AAC2AEF203C0B5F202C0B4F201C0B3F29F
:100D100000C0B2F279DE03C09CF202C09BF201C0B7
:100D20009AF200C099F29CC2ADF29BC2ACF29AC298
:100D3000ABF299C2AAF29CC2B1F29BC2B0F29AC2C3
:100D4000AFF299C2AEF20FDF03C0A8F202C0A7F261
:100D500001C0A6F200C0A5F2BC0E0201AD6F240EC8
:100D6000AC6F670EAB6F7D0EAA6FA8C2B1F2A7C2BF
:100D7000B0F2A6C2AFF2A5C2AEF20001F4DE00C02E
:100D8000AAF201C0ABF202C0ACF203C0ADF2D8923D
:100D900003C0B1F202C0B0F201C0AFF200C0AEF2C7
:100DA000E30E0201B56FE40EB46F900EB36F820EC6
:100DB000B26F0001EDDC03C0A0F202C09FF201C0DF
:100DC0009EF200C09DF2A0C2ADF29FC2ACF29EC2E4
:100DD000ABF29DC2AAF2A8C2B1F2A7C2B0F2A6C2FB
:100DE000AFF2A5C2AEF2BFDE00C0AAF201C0ABF204
:100DF00002C0ACF203C0ADF2D89203C0B1F202C09F
:100E0000B0F201C0AFF200C0AEF21C0E0201B56F2D
:100E1000870EB46F570EB36F830EB26F0001B8DC4C
:100E200003C0A0F202C09FF201C09EF200C09DF27A
:100E3000A0C2ADF29FC2ACF29EC2ABF29DC2AAF2BA
:100E4000A8C2B1F2A7C2B0F2A6C2AFF2A5C2AEF27A
:100E50008ADE00C0AAF201C0ABF202C0ACF203C04D
:100E6000ADF2D89203C0B1F202C0B0F201C0AFF24D
:100E700000C0AEF2AB0E0201B56FE10EB46F9E0E74
:100E8000B36F830EB26F000183DC03C0A0F202C017
:100E90009FF201C09EF200C09DF20201AD6BAC6BEF
:100EA000AB6B7F0EAA6FA8C2B1F2A7C2B0F2A6C206
:100EB000AFF2A5C2AEF2000156DE00C0AAF201C038
:100EC000ABF202C0ACF203C0ADF2D89203C0B1F2F3
:100ED00002C0B0F201C0AFF200C0AEF2B40E020127
:100EE000B56F2A0EB46F820EB36FB26F000150DC83
:100EF00003C0A4F202C0A3F201C0A2F200C0A1F29A
:100F0000A4C2ADF2A3C2ACF2A2C2ABF2A1C2AAF2D9
:100F1000A8C2B1F2A7C2B0F2A6C2AFF2A5C2AEF2A9
:100F200022DE00C0AAF201C0ABF202C0ACF203C0E4
:100F3000ADF2D89203C0B1F202C0B0F201C0AFF27C
:100F400000C0AEF2800E0201B56F3E0EB46F060E09
:100F5000B36F830EB26F00011BDC03C0A4F202C0AA
:100F6000A3F201C0A2F200C0A1F2A4C2ADF2A3C2DA
:100F7000ACF2A2C2ABF2A1C2AAF2A8C2B1F2A7C25D
:100F8000B0F2A6C2AFF2A5C2AEF2EDDD00C0AAF289
:100F900001C0ABF202C0ACF203C0ADF2D89203C004
:100FA000B1F202C0B0F201C0AFF200C0AEF2AB0EBF
:100FB0000201B56FE10EB46F9E0EB36F820EB26F79
:100FC0000001C8EC03F003C0A4F202C0A3F201C008
:100FD000A2F200C0A1F29CC2ADF29BC2ACF29AC2D6
:100FE000ABF299C2AAF2A0C2B1F29FC2B0F29EC205
:100FF000AFF29DC2AEF2B7DD00C0AAF201C0ABF203
:1010000002C0ACF203C0ADF203C0B1F202C0B0F254
:1010100001C0AFF200C0AEF2A4C2B5F2A3C2B4F2F6
:10102000A2C2B3F2A1C2B2F2EFDC03C0A0F202C0CE
:101030009FF201C09EF200C09DF2020E0201AB6F52
:10104000950EE96EABC2EAFF7E0EEF5CA96FA9BFF9
:1010500001D015D0000ED880A955AD6BAC6FACBFD8
:10106000AD07000163EC03F000C0A1F20150800A5B
:101070000201A26F02C0A3F203C0A4F211D0AD6BB3
:10108000A9C2ACF2ACBFAD07000163EC03F003C032
:10109000A4F202C0A3F201C0A2F200C0A1F20201B8
:1010A000A4C2ADF2A3C2ACF2A2C2ABF2A1C2AAF238
:1010B000180EB16F720EB06F310EAF6F7E0EAE6F45
:1010C000000151DDD892A0C2B1F29FC2B0F29EC21F
:1010D000AFF29DC2AEF203C0B5F202C0B4F201C0DD
:1010E000B3F200C0B2F2C8EC03F003C0A0F202C039
:1010F0009FF201C09EF200C09DF206D00201A06BDB
:101100009F6B9E6B9D6B00019DC200F09EC201F023
:101110009FC202F0A0C203F0000C8E0E006E02010E
:10112000A851005EA9C202F0AAC201F0028E0052CC
:1011300009E0D890025202E1015204E00232013289
:10114000002EF7D7A9AF05D0011E021E012AD8B480
:10115000022A0001000C99C2B1F298C2B0F297C203
:10116000AFF296C2AEF2180E0201B56F720EB46FF6
:10117000310EB36F7E0EB26F000146DC03C0ABF2DE
:1011800002C0AAF201C0A9F200C0A8F2C6DF01C0E5
:10119000A6F20201A79199C29DF298C29CF297C251
:1011A0009BF296C29AF299C2ADF298C2ACF297C283
:1011B000ABF296C2AAF2B16BB06BAF6BAE6B000133
:1011C0008BEC03F006E30201A781A66D9B51800A18
:1011D0009B6F0201A16BA06B9F6B9E6B020EA96FB0
:1011E0009E0EE96EA9C2EAFF7F0EA625EF6E9DC294
:1011F000B1F29CC2B0F29BC2AFF29AC2AEF2180E2C
:10120000B56F720EB46F310EB36F7E0EB26F000108
:1012100004EC05F000C0A8F201C0A9F202C0AAF2D5
:1012200003C0ABF20201AD6BA6C2ACF2ACBFAD071E
:10123000000163EC03F0D882ABC2B1F2AAC2B0F2F3
:10124000A9C2AFF2A8C2AEF203C0B5F202C0B4F2B6
:1012500001C0B3F200C0B2F2C8EC03F003C09DF2CB
:1012600002C09CF201C09BF200C09AF27C0E020107
:10127000AD6F880EAC6F590EAB6F720EAA6F9DC228
:10128000B1F29CC2B0F29BC2AFF29AC2AEF20001C0
:101290006ADC00C0A8F201C0A9F202C0AAF203C031
:1012A000ABF2D89203C0B1F202C0B0F201C0AFF20B
:1012B00000C0AEF2E00E0201B56F970EB46F260EBD
:1012C000B36F750EB26F0001C8EC03F003C0A5F256
:1012D00002C0A4F201C0A3F200C0A2F2A5C2ADF206
:1012E000A4C2ACF2A3C2ABF2A2C2AAF29DC2B1F2F6
:1012F0009CC2B0F29BC2AFF29AC2AEF234DC00C024
:10130000A8F201C0A9F202C0AAF203C0ABF2D892BF
:1013100003C0B1F202C0B0F201C0AFF200C0AEF241
:10132000C40E0201B56F1D0EB46F1E0EB36F780EA2
:10133000B26F0001C8EC03F003C0A5F202C0A4F232
:1013400001C0A3F200C0A2F2A5C2ADF2A4C2ACF2E9
:10135000A3C2ABF2A2C2AAF29DC2B1F29CC2B0F289
:101360009BC2AFF29AC2AEF2B3EC05F000C0A8F295
:1013700001C0A9F202C0AAF203C0ABF2D89203C026
:10138000B1F202C0B0F201C0AFF200C0AEF25E0E28
:101390000201B56F500EB46F630EB36F7A0EB26F69
:1013A0000001C8EC03F003C0A5F202C0A4F201C022
:1013B000A3F200C0A2F2A5C2ADF2A4C2ACF2A3C2D5
:1013C000ABF2A2C2AAF29DC2B1F29CC2B0F29BC221
:1013D000AFF29AC2AEF2B3EC05F000C0A8F201C0C1
:1013E000A9F202C0AAF203C0ABF2D89203C0B1F2D4
:1013F00002C0B0F201C0AFF200C0AEF21A0E02019C
:10140000B56FFE0EB46F750EB36F7C0EB26F000138
:10141000C8EC03F003C0A5F202C0A4F201C0A3F21D
:1014200000C0A2F2A5C2ADF2A4C2ACF2A3C2ABF25C
:10143000A2C2AAF29DC2B1F29CC2B0F29BC2AFF2AC
:101440009AC2AEF2B3EC05F000C0A8F201C0A9F256
:1014500002C0AAF203C0ABF2D89203C0B1F202C03C
:10146000B0F201C0AFF200C0AEF2180E0201B56FCB
:10147000720EB46F310EB36F7E0EB26F0001C8EC06
:1014800003F003C0A5F202C0A4F201C0A3F200C0A1
:10149000A2F29DC2ADF29CC2ACF29BC2ABF29AC268
:1014A000AAF2A5C2B1F2A4C2B0F2A3C2AFF2A2C224
:1014B000AEF2B3EC05F0D8920201B16BB06BAF6B3A
:1014C0007F0EAE6F03C0B5F202C0B4F201C0B3F23A
:1014D00000C0B2F20001C8EC03F0A1C2ADF2A0C29C
:1014E000ACF29FC2ABF29EC2AAF203C0B1F202C03C
:1014F000B0F201C0AFF200C0AEF2B3EC05F003C031
:10150000A1F202C0A0F201C09FF200C09EF202014F
:10151000A7A119D0B16BB06BAF6B7F0EAE6FA1C23C
:10152000B5F2A0C2B4F29FC2B3F29EC2B2F2000101
:1015300004EC05F003C0A1F202C0A0F201C09FF2CA
:1015400000C09EF202019EC200F09FC201F0A0C244
:1015500002F0A1C203F00001000C0201AD6BAC6B04
:10156000AB6BAA6B8CC2B1F28BC2B0F28AC2AFF283
:1015700089C2AEF200018BEC03F001E22FE18CC2D4
:1015800098F28BC297F28AC296F289C295F22EEC3B
:1015900006F090C2ADF28FC2ACF28EC2ABF28DC239
:1015A000AAF203C0B1F202C0B0F201C0AFF200C0B3
:1015B000AEF2B3EC05F000C091F201C092F202C0AD
:1015C00093F203C094F203C099F202C098F201C0F2
:1015D00097F200C096F2BFDD3BD03AD089C291F2BB
:1015E00002018A51800A926F8BC293F28CC294F2EC
:1015F0008CC298F28BC297F2966F89C295F2000165
:101600002EEC06F090C2ADF28FC2ACF28EC2ABF2FD
:101610008DC2AAF203C0B1F202C0B0F201C0AFF2B3
:1016200000C0AEF2B3EC05F000C092F201C093F23C
:1016300002C094F203C095F203C099F202C098F27E
:1016400001C097F200C096F286DD800E011A00D02C
:1016500051EF0BF0800E0201816F826B836B846B04
:10166000AD6B80C2ACF2ACBFAD07000163EC03F020
:1016700000C085F201C086F202C087F203C088F282
:1016800084C28CF283C28BF282C28AF281C289F256
:1016900003C090F202C08FF201C08EF200C08DF242
:1016A0005CD77FC2ADF27EC2ACF27DC2ABF27CC22F
:1016B000AAF203C0B1F202C0B0F201C0AFF200C0A2
:1016C000AEF2B3EC05F0C7EF0FF0B60E006E036A92
:1016D000026A016A0201805181118211831102E1C3
:1016E000006A0DD0D89001BE09D08037813782378B
:1016F0008337033602360136002EF4D7019E0001EF
:10170000D9EF0FF08E0E006E9FC201F09EC202F064
:10171000036A015209E102C001F0026A080E005E8C
:10172000015202E1006A08D0D89001BE04D002360E
:1017300001360006F9D7019E000C020199918DC275
:1017400092F28CC291F28BC290F28AC28FF28DC259
:10175000ADF28CC2ACF28BC2ABF28AC2AAF2B16B10
:10176000B06BAF6BAE6B00018BEC03F005E30201D5
:1017700099819051800A906F92C2ADF291C2ACF201
:1017800090C2ABF28FC2AAF20201B16BB06BAF6B29
:101790008E0EAE6F00018BEC03F001E217E192C2F6
:1017A000ABF291C2AAF290C2A9F28FC2A8F2B5DC44
:1017B00002C09FF201C09EF2A5DF03C096F202C0F4
:1017C00095F201C094F200C093F2CED092C2ADF275
:1017D00091C2ACF290C2ABF28FC2AAF2800E0201AB
:1017E000B16F960EB06F180EAF6F960EAE6F000110
:1017F0008BEC03F0D8A0B0D092C2B1F291C2B0F29B
:1018000090C2AFF28FC2AEF20201B56BB46BB36B94
:101810008E0EB26F000104EC05F003C0ABF202C003
:10182000AAF201C0A9F200C0A8F277DC02C098F2C7
:1018300001C097F292C2B1F291C2B0F290C2AFF27F
:101840008FC2AEF20201B56BB46BB36B8E0EB26F8A
:10185000000104EC05F000C09AF201C09BF202C046
:101860009CF203C09DF298C29FF297C29EF24ADF9B
:10187000D8829DC2B1F29CC2B0F29BC2AFF29AC2B2
:10188000AEF203C0B5F202C0B4F201C0B3F200C0C0
:10189000B2F2C8EC03F00201AD6BAC6BAB6B8E0E19
:1018A000AA6F03C0B1F202C0B0F201C0AFF200C033
:1018B000AEF20001B3EC05F003C092F202C091F267
:1018C00001C090F200C08FF298C29FF297C29EF2C0
:1018D00019DF0201AD6BAC6BAB6B8E0EAA6F03C050
:1018E000B1F202C0B0F201C0AFF200C0AEF200012E
:1018F000B3EC05F003C096F202C095F201C094F279
:1019000000C093F292C2ABF291C2AAF290C2A9F2C5
:101910008FC2A8F202DC02C09FF201C09EF2F2DE8A
:10192000D89296C2B1F295C2B0F294C2AFF293C20D
:10193000AEF203C0B5F202C0B4F201C0B3F200C00F
:10194000B2F2C8EC03F003C096F202C095F201C0F7
:1019500094F200C093F208D092C296F291C295F22E
:1019600090C294F28FC293F292C2ABF291C2AAF2E9
:1019700090C2A9F28FC2A8F28DEC08F002C09FF2CB
:1019800001C09EF2BFDED88292C2B1F291C2B0F223
:1019900090C2AFF28FC2AEF203C0B5F202C0B4F291
:1019A00001C0B3F200C0B2F2C8EC03F003C092F27F
:1019B00002C091F201C090F200C08FF2020199A121
:1019C00003D09451800A946F92C2ADF291C2ACF2EE
:1019D00090C2ABF28FC2AAF2B16BB06BAF6BAE6BC1
:1019E00000018BEC03F03CE0020199A11CD08E5366
:1019F0001AE1D88296C2B1F295C2B0F294C2AFF2A7
:101A000093C2AEF2B56BB46BB36B7F0EB26F0001D5
:101A1000C8EC03F003C096F202C095F201C094F244
:101A200000C093F2020199B11CD08E2D1AD0D89229
:101A300096C2B1F295C2B0F294C2AFF293C2AEF2C6
:101A4000B56BB46BB36B7F0EB26F0001C8EC03F0E3
:101A500003C096F202C095F201C094F200C093F266
:101A600002018DC2ADF28CC2ACF28BC2ABF28AC263
:101A7000AAF2B16BB06BAF6BAE6B00018BEC03F0F5
:101A800006E10201966B956B946B936B000193C218
:101A900000F094C201F095C202F096C203F05DEF2F
:101AA0000DF089C28DF288C28CF287C28BF286C299
:101AB0008AF202018E6B000140D616EF10F0010E83
:101AC00002017F5D006E000E8059016E000E81598B
:101AD000026E000E8259036E8A6B896B886B010E51
:101AE000876F00508B6F07E0D8908737883789372A
:101AF0008A378B2FF9D7866B856B846B836B865106
:101B0000825D43E30BE18551815D3FE307E1845151
:101B1000805D3BE303E17F51835D37E294908B80EE
:101B2000030E006E002EFED787517B15006E885184
:101B30007C15016E89517D15026E8A517E15036EEA
:101B4000005206E1015204E1025202E1035203E0B5
:101B500094928B8202D094928B92030E006E002E90
:101B6000FED794908B90030E006E002EFED7D89077
:101B70008A33893388338733010E8327D8B0842B87
:101B8000D8B4852BD8B4862BBAD70001000C02013B
:101B9000766B74530FE173530DE1725104080AE33D
:101BA00003E171510E0806E3746B736B040E726FE0
:101BB0000F0E716F74530AE1735308E172510308F9
:101BC00012E2FF0A03E171510E080DE274530BE1BA
:101BD000735309E17251080806E303E171511B08D0
:101BE00002E3766BC5D174530AE1735308E1725175
:101BF000070813E2FF0A03E171511B080EE2745358
:101C00000CE173530AE17251100807E303E17151CB
:101C1000370803E3010E766FABD174530AE17353B7
:101C200008E172510F0813E2FF0A03E1715137080E
:101C30000EE274530CE173530AE17251200807E37A
:101C400003E171516F0803E3020E766F91D1745373
:101C50000AE1735308E172511F0813E2FF0A03E11E
:101C600071516F080EE274530CE173530AE1725123
:101C7000400807E303E17151E10803E3030E766FC7
:101C800077D174530AE1735308E172513F0813E2AC
:101C9000FF0A03E17151E1080EE274530CE1735342
:101CA0000AE17251810807E303E17151C30803E3BC
:101CB000040E766F5DD174530AE1735308E17251DB
:101CC000800815E2FF0A03E17151C30810E2745362
:101CD0000EE1735101080BE307E17251030807E3BA
:101CE00003E171517D0803E3050E766F41D1745312
:101CF0000DE1735100081AE2FF0A08E1725102086F
:101D000015E2FF0A03E171517D0810E274530EE100
:101D1000735102080BE307E17251070807E303E17F
:101D20007151230803E3060E766F22D174530DE13F
:101D3000735101081AE2FF0A08E17251060815E220
:101D4000FF0A03E17151230810E274530EE173514D
:101D500004080BE307E172510D0807E303E1715139
:101D6000E30803E3070E766F03D174530DE173515B
:101D700003081AE2FF0A08E172510C0815E2FF0A93
:101D800003E17151E30810E274530EE17351080846
:101D90000BE307E172511B0807E303E17151C70828
:101DA00003E3080E766FE4D074530DE17351070816
:101DB0001AE2FF0A08E172511A0815E2FF0A03E16C
:101DC0007151C70810E274530EE1735110080BE310
:101DD00007E17251380807E303E17151570803E343
:101DE000090E766FC5D074530DE173510F081AE2D6
:101DF000FF0A08E17251370815E2FF0A03E1715149
:101E0000570810E274530EE1735120080BE307E109
:101E10007251700807E303E17151AF0803E30A0E42
:101E2000766FA6D074530DE173511F081AE2FF0AB2
:101E300008E172516F0815E2FF0A03E17151AF0822
:101E400010E274530EE1735140080BE307E1725145
:101E5000E10807E303E171515F0803E30B0E766FBE
:101E600087D074530DE173513F081AE2FF0A08E16D
:101E70007251E00815E2FF0A03E171515F0810E2B8
:101E800074530EE1735181080BE307E17251BE08F0
:101E900007E303E17151D70803E30C0E766F68D0B6
:101EA00074530DE1735180081CE2FF0A08E172517E
:101EB000BD0817E2FF0A03E17151D70812E274511D
:101EC00001080FE30BE1735103080BE307E17251C3
:101ED0008D0807E303E171514F0803E30D0E766FA0
:101EE00047D07451000821E2FF0A0DE17351020846
:101EF0001CE2FF0A08E172518C0817E2FF0A03E1B5
:101F000071514F0812E2745102080FE30BE1735153
:101F100006080BE307E17251F30807E303E171518F
:101F20008F0803E30E0E766F23D07451010820E270
:101F3000FF0A0DE1735105081BE2FF0A08E1725127
:101F4000F20816E2FF0A03E171518F0811E27451A1
:101F500004080EE30BE173510E080AE307E1725126
:101F60000E0806E303E171512F0802E30F0E766FAE
:101F70000A0E76257B6F7F6BE00E7E6F010E7D6F04
:101F80008A0E7C6F7BC280F200012AEF0BF000C04A
:101F90007CF201C07DF202C07EF203C07FF274C207
:101FA00083F273C282F272C281F271C280F265EF73
:101FB0000BF07FC2B1F27EC2B0F27DC2AFF27CC242
:101FC000AEF203C0B5F202C0B4F201C0B3F200C079
:101FD000B2F204EC05F0EACF81F2E9CF80F2D882C8
:101FE0000201B16BB06BAF6B8A0EAE6F03C0B5F27E
:101FF00002C0B4F201C0B3F200C0B2F20001C8ECFA
:1020000003F081C2EAFF80C2E9FF00C082F201C092
:1020100083F202C084F203C085F203C089F202C0D9
:1020200088F201C087F200C086F23BD503C0ABF254
:1020300002C0AAF201C0A9F200C0A8F28DEC08F01B
:1020400002C07AF201C079F20201763BF00E7617F7
:1020500079377A3779377A37FC0E79177B6B7A5173
:102060000F0B776F765177137951FC0B786F7551A1
:1020700078137E6B7D6B7C6B77C27BF2826B816B9E
:10208000806B080E7F6F00011ADD02017E6B7D6B95
:102090007C6B78C27BF2826B816B806B080E7F6FEA
:1020A00000010DDD000C94908B8002016C51000149
:1020B00007E0010A21E0030A3BE0010A55E070D085
:1020C000969A8D9A100E006E002EFED7000070C2F8
:1020D00074F26FC273F26EC272F26DC271F2020ECE
:1020E0000201756F000153DD100E006E002EFED749
:1020F0000000969A8D8A55D096988D98100E006E95
:10210000002EFED7000070C274F26FC273F26EC26E
:1021100072F26DC271F2020E0201756F000137DDBD
:10212000100E006E002EFED7000096988D8839D0D4
:1021300096968D96100E006E002EFED7000070C28F
:1021400074F26FC273F26EC272F26DC271F2020E5D
:102150000201756F00011BDD100E006E002EFED710
:10216000000096968D861DD096948D94100E006E6C
:10217000002EFED7000070C274F26FC273F26EC2FE
:1021800072F26DC271F2020E0201756F0001FFDC86
:10219000100E006E002EFED7000096948D8401D0A4
:1021A00000D094908B90000C0201B151000107E027
:1021B000010A27E0030A47E0010A67E088D002012C
:1021C000B251FC0F1DE2040F00016BEF11F0979C60
:1021D0008E9C979E8E9E020113D0979C8E8C979E0C
:1021E0008E9E02010DD0979C8E9C979E8E8E020132
:1021F00007D0979C8E8C979E8E8E020101D0020193
:1022000068D00201B251FC0F1DE2040F000181EF02
:1022100011F097988E98979A8E9A020113D09798FA
:102220008E88979A8E9A02010DD097988E98979AD9
:102230008E8A020107D097988E88979A8E8A02011B
:1022400001D0020146D00201B251FC0F1DE2040F81
:10225000000197EF11F097948E9497968E96020155
:1022600013D097948E8497968E9602010DD09794F2
:102270008E9497968E86020107D097948E849796B7
:102280008E86020101D0020124D00201B251FC0F5E
:102290001DE2040F0001ADEF11F097908E90979220
:1022A0008E92020113D097908E8097928E920201A7
:1022B0000DD097908E9097928E82020107D09790C2
:1022C0008E8097928E82020101D0020102D002011B
:1022D00000D00001000CF2CF0EF0F29EE824F76A65
:1022E000F736FB0FF66E220EF7220A00F550FA6E53
:1022F0000800F5500EBEF28EF96ECE21DA21E621ED
:10230000F221F2CF0EF0F29EE824F76AF736270F9B
:10231000F66E230EF7220A00F550FA6E0800F5500B
:102320000EBEF28EF96E12221E222A223622F2CF21
:102330000EF0F29EE824F76AF736530FF66E230E7E
:10234000F7220A00F550FA6E0800F5500EBEF28E24
:10235000F96E562262226E227A22F2CF0EF0F29E9F
:10236000E824F76AF7367F0FF66E230EF7220A008D
:10237000F550FA6E0800F5500EBEF28EF96E9A22F4
:10238000A622B222BE220201B151000107E0010AD9
:1023900013E0030A1FE0010A2BE038D00201B2511A
:1023A000000103E0010A04E006D093948A9403D06C
:1023B00093948A8400D02BD00201B251000103E033
:1023C000010A04E006D093968A9603D093968A86F3
:1023D00000D01DD00201B251000103E0010A04E067
:1023E00006D093988A9803D093988A8800D00FD00B
:1023F0000201B251000103E0010A04E006D0939A01
:102400008A9A03D0939A8A8A00D001D000D0000C17
:1024100002013F6B010131950001000C020E020127
:10242000B05F0CE3020EEA6EB00EE96EEF5006E00C
:10243000020E006E002EFED7EF2EFAD70001000C20
:10244000186AF2BE188EF29E21EC01F018BEF28ED0
:1024500002C0B1F201C0B0F20201B1BF0CD0B15163
:102460001B0809E2FF0A03E1B051200804E21C0E38
:10247000B16F200EB06FB1AF0BD0B151E30808E3DC
:1024800003E1B051DF0804E3E30EB16FE00EB06F7B
:10249000B0C201F0B1C202F00001000C0201BD5156
:1024A000C119800BC76FBDAF0BD0BA1FBB1FBC1FBC
:1024B000BD1FBA2BD8B4BB2BD8B4BC2BD8B4BD2B02
:1024C000C1AF0BD0BE1FBF1FC01FC11FBE2BD8B4D2
:1024D000BF2BD8B4C02BD8B4C12B006A016A026AE2
:1024E000036AC26BC36BC46BC56BC151C011BF1112
:1024F000BE112CE0200EC66FD890BA37BB37BC3760
:10250000BD37C237C337C437C537C151C55D08E1D0
:10251000C051C45D05E1BF51C35D02E1BE51C25D62
:102520000FE3BE51C25FBF51D8A0BF3DC35FC051D2
:10253000D8A0C03DC45FC151D8A0C13DC55FD880FF
:102540000036013602360336C62FD6D7C7AF0BD0BA
:10255000001E011E021E031E002AD8B4012AD8B490
:10256000022AD8B4032A020EEA6EC20EE96E0001F6
:10257000D4EF13F002019B6B9A6B996B100E986F5E
:10258000966B9651030809E396C2B1F295C2B2F276
:1025900000010ADE0201962BF4D7020EB06FFA0E8C
:1025A000B16F00012DEC02F00201B02FF8D7966B4D
:1025B000965103080FE39651040DF350036A9C0FE4
:1025C000E96E020E0320EA6EEF6AEC6AEC6AEC6ACE
:1025D000962BEED7966B96510308D8A0F5D0976B43
:1025E000975101082AE3186AF2BE188EF29E96C22D
:1025F000C9F2CA6B00015EEC01F018BEF28E640EE7
:102600000201B06F00010ADF968C84BCFDD718DF91
:1026100001C000F002C001F0026A036A01AE02D0FC
:102620000206030603C0AFF202C0AEF201C0ADF273
:1026300000C0ACF20201972BD3D7976B97AF03D0B2
:102640009BAF0CD002D09BBF6CD09B5307E19A5339
:1026500005E1995303E19851975D63E2186AF2BE70
:10266000188EF29E96C2C9F2CA6B00015EEC01F0B0
:1026700018BEF28E640E0201B06F0001CFDE968CA0
:1026800084BCFDD7DDDE01C000F002C001F0026AAB
:10269000036A01AE02D00206030603C0AFF202C015
:1026A000AEF201C0ADF200C0ACF202019651040DD1
:1026B000F350036A9C0F016E020E032201C0B0F2B8
:1026C00003C0B1F29651040DF350036A9C0FE96EFA
:1026D000020E0320EA6EEFCFB2F2ECCFB3F2ECCFF2
:1026E000B4F2ECCFB5F2AC51B225006EAD51B321CE
:1026F000016EAE51B421026EAF51B521B1C2EAFFF5
:10270000B0C2E9FF00C0EFFF01C0ECFF02C0ECFF68
:10271000EC6E0A0EB16F00012DEC02F00201972B56
:102720008DD796A103D09298899802D092988988E3
:102730009651080DF350B16BB06FD8909535036A80
:10274000B025016EB151032201504E0F016E010EF2
:10275000032201C0B2F203C0B3F29651040DF3504C
:10276000036A9C0FE96E020E0320EA6EEFCFB4F20B
:10277000ECCFB5F2ECCFB6F2ECCFB7F2EACFB9F2CC
:10278000E9CFB8F2B7C2BDF2B6C2BCF2B5C2BBF275
:10279000B4C2BAF29BC2C1F29AC2C0F299C2BFF2ED
:1027A00098C2BEF200017AD6B9C2EAFFB8C2E9FF08
:1027B000B3C2EAFFB2C2E9FF01C0ECFFED5200C0B4
:1027C000EFFF0201962B07D7966B9651030822E381
:1027D000036A9651460FE96E010E0320EA6EEFCFB1
:1027E000B0F296C2B1F2B0C2B2F20001DDDC036A0F
:1027F000020196514A0FE96E010E0320EA6EEFCFF7
:10280000B0F296C2B1F2B0C2B2F20001BCDD020178
:10281000962BDBD700017DEF14F0100E0201946FB0
:102820006C5302E0040E946FF29CF29EF2BEFDD750
:1028300098948F946E6B6E5107080FE3FA0EB16F88
:1028400000012DEC02F002016EA103D0929889984C
:1028500002D0929889886E2BEED76D6B6D5103086C
:102860003DE36F6B6F51030837E36F51080DF35071
:10287000966B956FD8906D35036A9525016E9651CC
:1028800003220150700F016E020E032201C097F265
:1028900003C098F26F51080DF3509A6B996FD8905E
:1028A0006D35036A9925016E9A51032201504E0F2E
:1028B000E96E010E0320EA6EECCF03F0ED52EFCF8C
:1028C0009BF298C2EAFF97C2E9FF03C0ECFFED520A
:1028D0009BC2EFFF6F2BC6D76D2BC0D76D6B6D51B1
:1028E0000308D8A0EED0010E906F936B9053D8B42C
:1028F000E6D06DC295F200013DD60201932B906B9C
:102900006F6B6F510308D8A0D5D06F51080DF350ED
:10291000966B956FD8906D35036A9525016E96512B
:10292000032201504E0FE96E010E0320EA6EECCF38
:1029300098F2ED52EFCF97F26F51080DF3509A6B6A
:10294000996FD8906D35036A9925016E9A510322CB
:102950000150700FE96E020E0320EA6EECCF03F017
:10296000ED52EF50975D916F03509859926F92BF5F
:1029700005D0925366E19151140863E392AF07D0FA
:102980009251FF0804E35DE19151EB085AE26F5167
:10299000080DF350966B956FD8906D35036A9525A9
:1029A000016E9651032201504E0FE96E010E032075
:1029B000EA6EECCF98F2ED52EFCF97F298C203F0A7
:1029C000975198AF08D0000ED8809755006E000E32
:1029D0009855036E0050986F03C099F298512008E3
:1029E00003E199511C082DE06F51080DF3509B6BCA
:1029F0009A6FD8906D35036A9A25016E9B51032218
:102A00000150700FE96E020E0320EA6EECCF9DF2CA
:102A1000ED52EFCF9CF29DC203F09C519DAF08D0C8
:102A2000000ED8809C55006E000E9D55036E005020
:102A30009D6F03C09EF29D51200805E19E511C0828
:102A400002E1010E906F6F51080DF350966B956F78
:102A5000D8906D35036A9525016E96510322015079
:102A6000700F016E020E032201C097F203C098F2AC
:102A70006F51080DF3509A6B996FD8906D35036ABA
:102A80009925016E9A51032201504E0FE96E010EF5
:102A90000320EA6EECCF03F0ED52EFCF9BF298C229
:102AA000EAFF97C2E9FF03C0ECFFED529BC2EFFFC4
:102AB0006F2B27D79351945D01E2906B17D76D2B45
:102AC0000ED79298898898948F84C00EF2120001D4
:102AD000000CB0989484BD6A796A9482BA6A676A75
:102AE000C150C00B0D09C16EC080C082C084C08EB1
:102AF000C280000E016EC250C30B0110C26E08EFFF
:102B000002F001017E6B7E5303E0949C8B8C02D01B
:102B1000949C8B9C929A899A948E7C6B82BE7C2B1F
:102B20007CC17DF1020E02015D6FFA0EB16F0001F2
:102B30002DEC02F002015D2FF8D70101776BFA0E40
:102B4000766FB50ECD6E480E0509CA6EF90ECB6EC6
:102B5000020E02016D6F400E6C6F000142EC02F03C
:102B6000C69A949A94889496310EC66E400EC76E9B
:102B7000C76A8FEF02F046EF03F0030E0101466FC4
:102B80004A6B476B4B6B020E486F4C6B496B4D6B3E
:102B9000396B386B040E376F4C0E366F3D6B3C6BE8
:102BA000130E3B6F880E3A6F416B406B4E0E3F6FBA
:102BB000200E3E6F456B446B130E436F880E426FC1
:102BC00002015B6B5B510308D8A0B0D0D8905B3595
:102BD000036A6E0FE96E010E0320EA6EEC6AED5295
:102BE000EF6A036A5B51320FE96E010E0320EA6E51
:102BF000EF6A5B51040DF350036A360FE96E010E64
:102C00000320EA6EEFCF5DF2ECCF5EF2ECCF5FF225
:102C1000ECCF60F25BC26CF260C270F25FC26FF226
:102C20005EC26EF25DC26DF2000153EC10F0036AF9
:102C300002015B51460FE96E010E0320EA6EEFCFF1
:102C40005DF25BC2B1F25DC2B2F20001D4EC10F0F1
:102C5000036A02015B514A0FE96E010E0320EA6E1E
:102C6000EFCF5DF25BC2B1F25DC2B2F20001C3EC24
:102C700011F002015B51080DF3505E6B5D6F190E90
:102C80005D25E96E000E5E21EA6E010EEF6E5B516E
:102C9000080DF3505E6B5D6F010E5D25016E000E39
:102CA0005E21036E0150190FE96E000E0320EA6EDB
:102CB000010EEF6E5B51080DF3505E6B5D6F020EFF
:102CC0005D25016E000E5E21036E0150190FE96E45
:102CD000000E0320EA6EEF6A5B51080DF3505E6B45
:102CE0005D6F030E5D25016E000E5E21036E0150C7
:102CF000190FE96E000E0320EA6EEF6A5B51080DB2
:102D0000F3505E6B5D6F060E5D25016E000E5E2159
:102D1000036E0150190FE96E000E0320EA6E010EDA
:102D2000EC6EED52400EEF6E5B2B4CD7186AF2BE84
:102D3000188EF29EC96B32C1CAF200015EEC01F03E
:102D400018BEF28E0101306B000108EC12F0969271
:102D50008D8296908D8001012F6B2E6B2D6B2C6BCD
:102D60002B6B2A6B296B796B010E786F7B6B7A6FFB
:102D70009D80C00EF2129298898802016C6B00014E
:102D80004CDD92988998FDEF24F057C2EAFF56C2B5
:102D9000E9FF020174C2EFFFE92AD8B4EA2AEF6A18
:102DA000562BD8B4572B0001000C020173BF11D071
:102DB0000F0E006E723900160A0E005C03E2300E30
:102DC000002602D07351002600C074F20001DDDF3E
:102DD00002010F0E72170A0E725D02E2300E02D06F
:102DE000739F7351722772C274F20001CEDF000C20
:102DF00002016F6B6F5177080BE3036A6F51C20FCB
:102E0000E96E010E0320EA6EFF0EEF6E6F2BF2D714
:102E10006CC200F06D51036E05E100520001D8B4A0
:102E200072D00201035006E1010E005C0001D8B42B
:102E30007BD00201035006E1020E005C0001D8B411
:102E400085D00201035006E1030E005C0001D8B4F6
:102E50008FD00201035006E1040E005C0001D8B4DB
:102E600099D00201035006E1050E005C0001D8B4C0
:102E7000AAD00201035006E1060E005C0001D8B49E
:102E8000C4D00201035006E1070E005C0001D8B473
:102E9000D5D00201035006E1080E005C0001D8B451
:102EA000DFD00201035006E1090E005C0001D8B436
:102EB000FBD00201035006E10A0E005C0001D8B409
:102EC00013D10201035006E10B0E005C0001D8B4DF
:102ED0002BD10201035006E10C0E005C0001D8B4B6
:102EE00042D10201800E035C05E100520001D8B41A
:102EF00069D10201035006E1800E005C0001D8B4E4
:102F000073D102018ED1010E0201576FC20E566FAE
:102F1000726B370E736F000148DF0201726B370E60
:102F2000736F000142DF8ED1010E0201576FC20E96
:102F3000566F726B370E736F000137DF010E02019F
:102F4000726F370E736F000130DF7CD1010E02010A
:102F5000576FC20E566F726B370E736F000125DF0D
:102F6000020E0201726F370E736F00011EDF6AD10D
:102F7000010E0201576FC20E566F726B370E736FE0
:102F8000000113DF030E0201726F370E736F000131
:102F90000CDF58D1010E0201576FC20E566F726BD3
:102FA000370E736F000101DF040E0201726F370EDE
:102FB000736F0001FADE6EC272F2370E0201736F98
:102FC0000001F3DE3FD1010E0201576FE40E566F90
:102FD000010E726F370E736F0001E7DE0201726B34
:102FE000370E736F0001E1DE020E0201706F300ECA
:102FF000746F0001CADE0201702FF9D7060E726FDE
:10300000370E736F0001D1DE1DD1010E0201576F23
:10301000C20E566F726B370E736F0001C6DE060E5E
:103020000201726F370E736F0001BFDE6EC272F263
:10303000370E0201736F0001B8DE04D1010E0201E8
:10304000576FC20E566F726B370E736F0001ADDE95
:10305000070E0201726F370E736F0001A6DEF2D009
:10306000010E0201576FC20E566F726B370E736FEF
:1030700000019BDE080E0201726F370E736F0001B4
:1030800094DE050E0201706F705100010FEC01F02B
:103090000201702B006E746F000177DE090E0201D1
:1030A000705DF2E10001CED0010E0201576FC20E39
:1030B000566F726B370E736F000177DE090E0201D7
:1030C000726F370E736F000170DE7BC172F2370EC4
:1030D0000201736F000169DE7AC172F2370E0201DC
:1030E000736F000162DEAED0010E0201576FC20E97
:1030F000566F726B370E736F000157DE0A0E0201B6
:10310000726F370E736F000150DE7BC172F2370EA3
:103110000201736F000149DE7AC172F2370E0201BB
:10312000736F000142DE8ED0010E0201576FC20E96
:10313000566F726B370E736F000137DE0B0E020194
:10314000726F370E736F000130DE0201726B370E43
:10315000736F00012ADE780E0201726F370E736FF3
:10316000000123DE6FD0010E0201576FC20E566FB1
:10317000020E706F300E746F000107DE0201702FB7
:10318000F9D70C0E726F370E736F00010EDE010E51
:103190000201726F370E736F000107DE0201726B5E
:1031A000370E736F000101DE0201726B370E736F11
:1031B0000001FBDD060E0201726F370E736F000116
:1031C000F4DD40D0010E0201576FC20E566F800E23
:1031D000726F370E736F0001E8DD0201726B370EFC
:1031E000736F0001E2DD2ED0010E0201576FC20E97
:1031F000566F020E706F300E746F0001C6DD020153
:10320000702FF9D7800E726F370E736F0001CDDD0E
:103210007CC172F2370E0201736F0001C6DD12D05D
:103220000201010E576FC20E566F726B370E736F2D
:103230000001BBDD040E0201726F370E736F0001D7
:10324000B4DD00D0000C71C273F270C272F273C2AE
:1032500003F0020172C2E9FF73C2EAFFEF5206E017
:10326000722BD8B4732B0001F2D702017051725D3A
:10327000006E71517359036E00C001F0026E0001BF
:103280004BEF19F002016F6B6E6B010E716FC20E86
:10329000706F0001D8D702C003F00150035205E15E
:1032A000015002016E5D0DE20001036A02016E51E0
:1032B000C20FE96E010E0320EA6EEF506F276E2BEE
:1032C000E4D76F1F6FC201F00001ADEF19F0640E7B
:1032D0000201716F988086A004D0715302E07107DB
:1032E000F9D77051F2CF72F2F29E000182EC00F039
:1032F000020172BFF28E956A8C6E96908D9000D00E
:1033000096908D800001000C02016FBF11D00F0E4E
:10331000006E6E3900160A0E005C03E2300E0026C5
:1033200002D06F51002600C070F20001D0DF020110
:103330000F0E6E170A0E6E5D02E2300E02D06F9F06
:103340006F516E276EC270F20001C1DFD6EF19F027
:1033500002016C6B6D6B000195D701C06DF2020E1E
:103360000201706F0001B3DF036A02016C51C20FEA
:10337000E96E010E0320EA6EEF5212E0036A6C510F
:10338000C20FE96E010E0320EA6EEFCF6EF26EC23D
:1033900070F200019CDF02016C2B0001E5D70201F5
:1033A0006DC26EF2370E6F6F0001AED7030E0201D1
:1033B000706F00018CDF000C0201606B988286B296
:1033C00016D096928D92060E006E002EFED700004B
:1033D000FF0E956E8350F2CF62F2F29E000182ECF6
:1033E00000F0020162BFF28E606F96928D8260C221
:1033F00001F00001D2EF1AF00201726B736B746B73
:10340000756B716B7051715D5EE272377337743733
:103410007537723773377437753772377337743758
:1034200075377237733774377537F00E7217036A52
:1034300071516E25E96E6F510320EA6EEF50390825
:1034400020E3036A71516E25E96E6F510320EA6E25
:10345000EF507225766F000E7321776F000E742186
:10346000786F000E7521796F300E765D726F000EE9
:103470007759736F000E7859746F000E7959756F14
:1034800020D00A0E7225766F000E7321776F000E22
:103490007421786F000E7521796F036A71516E2562
:1034A000E96E6F510320EA6E410EEF5C7625726F74
:1034B000000E7721736F000E7821746F000E792152
:1034C000756F712B9FD772C200F073C201F074C286
:1034D00002F075C203F00001000C02015E6B5F6B2D
:1034E00001018251020803E0000E016E42D0010E7C
:1034F00002013E5D036A820FE96E010E0320EA6E4F
:10350000EF50030805E0000E016E010132D0020108
:10351000010E606F030E3E5D605D0BE2036A605159
:10352000820FE96E010E0320EA6EEF505E27602BDA
:10353000F1D75E1F030E3E5D036A820F636F010EBB
:103540000320646F6F6F63C26EF2020E706F000132
:1035500053DF00C05FF202015E515F5D06E0000EC6
:10356000016E010106D005D00201010E016E0101BC
:1035700000D00001F6EF1AF008EC12F002015D6BCA
:103580005D513F0827E3988286B221D0036A5D51DE
:10359000820F016E010E032201C05EF203C05FF2D2
:1035A00000010AD75FC2EAFF5EC2E9FF01C0EFFF78
:1035B000036A02015D51820FE96E010E0320EA6E7B
:1035C000EF50030803E15DC23FF204D001D002D006
:1035D0005D2BD6D73F513F0814E3010131B50FD021
:1035E000010E02013F253E6F000177D7015204E032
:1035F0000101318504D0000108EC12F0010105D071
:103600000201000108EC12F00101000129EF25F090
:10361000D56ACD6A08EC12F09D9AF29AF29CF29E5D
:10362000F2BEFDD724EF1DF06DC277F16CC276F1CA
:10363000010176C100F07751036E05E17D0E005C5B
:10364000000121E00101035005E1FA0E005C0001D8
:1036500024E00101010E035C05E1F40E005C0001B1
:1036600026E00101030E035C05E1E80E005C0001A9
:1036700029E00101070E035C05E1D00E005C0001AA
:103680002CE001010AD00101776B7D0E766F480EA8
:103690000609CA6E7C0ECB6E2BD00101776BFA0E39
:1036A000766F480E0509CA6EF90ECB6E21D0010E59
:1036B0000101776FF40E766F480E0509CA6E7C0E15
:1036C000CB6E16D0030E0101776FE80E766F480EB1
:1036D0000409CA6EF90ECB6E0BD0070E0101776F8D
:1036E000D00E766F480E0409CA6E7C0ECB6E00D0E9
:1036F0000001DBEF1DF0016A026A006A036A020141
:10370000755102E1745118E0100E766FD89072373F
:103710007337003603367551035C02E17451005C67
:1037200007E37451005ED8A003067551035ED8808C
:1037300001360236762FEAD70001C0EF22F09298C8
:103740008988010E02016F6F830E6E6F040E706F19
:10375000000152DE01C05CF200C05BF202015BC2FC
:1037600000F05C51036E06E1020E005C0001D8B46B
:103770003ED10201035006E1030E005C0001D8B403
:1037800041D10201035006E1070E005C0001D8B4EC
:103790004BD10201035006E1050E005C0001D8B4D4
:1037A0005DD10201035006E1060E005C0001D8B4B1
:1037B00060D10201035006E1080E005C0001D8B49C
:1037C00085D10201035006E1090E005C0001D8B466
:1037D00095D10201035006E10C0E005C0001D8B443
:1037E000A5D10201035006E1640E005C0001D8B4CB
:1037F000A8D10201035006E1650E005C0001D8B4B7
:10380000C8D10201035006E1660E005C0001D8B485
:10381000EAD10201035006E1670E005C0001D8B452
:1038200016D20201035006E1680E005C0001D8B414
:103830004FD20201035006E1690E005C0001D8B4CA
:103840009CD20201035006E16A0E005C0001D8B46C
:10385000E9D20201035006E16B0E005C0001D8B40E
:1038600016D30201035006E16C0E005C0001D8B4CF
:103870004FD30201035006E16D0E005C0001D8B485
:103880007CD30201035006E16E0E005C0001D8B447
:10389000BBD30201035007E16F0E005C0001D8B4F6
:1038A0002CEF20F00201035007E1700E005C0001D4
:1038B000D8B45AEF20F00201035007E1710E005C0A
:1038C0000001D8B4A0EF20F00201035007E1720E0E
:1038D000005C0001D8B40BEF21F00201035007E1B6
:1038E000730E005C0001D8B439EF21F002010350DF
:1038F00007E1740E005C0001D8B43FEF21F0020133
:10390000035007E1750E005C0001D8B49AEF21F076
:103910000201035007E1760E005C0001D8B4F0EF1D
:1039200021F00201035007E1770E005C0001D8B4DA
:103930001CEF22F00201035007E1780E005C000149
:10394000D8B440EF22F00201035007E1790E005C89
:103950000001D8B4EDEF22F00201035007E17B0E25
:10396000005C0001D8B44BEF23F00201035007E1E3
:103970007A0E005C0001D8B489EF23F002010350F5
:1039800007E17C0E005C0001D8B4DCEF23F00201FB
:10399000035007E17D0E005C0001D8B408EF24F06D
:1039A0000201035007E17E0E005C0001D8B427EF4E
:1039B00024F00201035007E17F0E005C0001D8B43F
:1039C00046EF24F00201035007E1810E005C000184
:1039D000D8B469EF24F00201035007E1820E005CC5
:1039E0000001D8B469EF24F002016AEF24F002016B
:1039F0006D6B020E6C6F6E6B0001F8EC16F0A8DCBC
:103A000074EF24F002016D6B030E6C6F6E6B00019E
:103A1000F8EC16F09DDC640E0201B16F00012DEC94
:103A200002F0FF0074EF24F0F29CF29EF2BEFDD78C
:103A300002016D6B070E6C6F6E6B0001F8EC16F0F7
:103A400087DC08EC12F0E4D5640E0201B16F0001CE
:103A50002DEC02F000EF5BF074EF24F002016D6BCF
:103A6000050E6C6F6E6B0001F8EC16F071DC74EFF4
:103A700024F0010E02016F6F870E6E6F020E706FE1
:103A80000001BADC005206E1015204E1025202E1F7
:103A900003520DE0010E01012F6F020E02016D6F46
:103AA000400E6C6F000142EC02F09D8203D00101D8
:103AB0002F6B9D9202016D6B060E6C6F2FC16EF223
:103AC0000001F8EC16F044DC74EF24F0010E020162
:103AD0006F6F870E6E6F040E706F00018DDC01C07A
:103AE0005CF200C05BF202016D6B080E6C6F6E6BD6
:103AF0000001F8EC16F02CDC74EF24F0010E02014A
:103B00006F6F870E6E6F040E706F000175DC01C061
:103B10005CF200C05BF202016D6B090E6C6F6E6BA4
:103B20000001F8EC16F014DC74EF24F002016D6B68
:103B30000C0E6C6F6E6B0001F8EC16F009DC74EF84
:103B400024F0010E0201576FC20E566F5CC272F272
:103B5000370E736F0001D5EC16F05BC272F2370EB0
:103B60000201736F0001D5EC16F077C172F2370EC7
:103B70000201736F0001D5EC16F076C172F2370EB8
:103B80000201736F0001D5EC16F0A8EC19F074EF88
:103B900024F0010E02016F6F870E6E6F040E706FBE
:103BA00000012ADC01C077F100C076F177C16DF227
:103BB00076C16CF239D5010E0201576FC20E566FF5
:103BC0005CC272F2370E736F0001D5EC16F05BC267
:103BD00072F2370E0201736F0001D5EC16F0A8ECFB
:103BE00019F074EF24F0010E02016F6F870E6E6FF3
:103BF000020E706F000100DC00C05DF2036A02017A
:103C00005D51460FE96E010E0320EA6EEFCF6CF2B4
:103C1000010E576FC20E566F5CC272F2370E736F91
:103C20000001D5EC16F05BC272F2370E0201736F21
:103C30000001D5EC16F06CC272F2370E0201736F00
:103C40000001D5EC16F0A8EC19F074EF24F0010E89
:103C500002016F6F870E6E6F020E706F0001FCEC39
:103C600019F000C05DF2010E02016F6F890E6E6FD8
:103C7000020E706F0001FCEC19F000C061F2036AE3
:103C800002015D51460FE96E010E0320EA6E61C22A
:103C9000EFFF5DC2B1F261C2B2F20001D4EC10F0EC
:103CA000010E0201576FC20E566F5CC272F2370EE0
:103CB000736F0001D5EC16F05BC272F2370E020191
:103CC000736F0001D5EC16F0A8EC19F074EF24F036
:103CD000010E02016F6F870E6E6F020E706F000192
:103CE000FCEC19F000C05DF202015D51040DF350CF
:103CF000036A360FE96E010E0320EA6EEFCF6CF215
:103D0000ECCF6DF2ECCF6EF2ECCF6FF2010E576F8D
:103D1000C20E566F5CC272F2370E736F0001D5ECA3
:103D200016F05BC272F2370E0201736F0001D5EC20
:103D300016F06FC272F2370E0201736F0001D5ECFC
:103D400016F06EC272F2370E0201736F0001D5ECED
:103D500016F06DC272F2370E0201736F0001D5ECDE
:103D600016F06CC272F2370E0201736F0001D5ECCF
:103D700016F0A8EC19F074EF24F0010E02016F6F39
:103D8000870E6E6F020E706F0001FCEC19F000C020
:103D90005DF2010E02016F6F890E6E6F080E706F7B
:103DA0000001FCEC19F003C065F202C064F201C02E
:103DB00063F200C062F202015D51040DF350036A28
:103DC000360FE96E010E0320EA6E62C2EFFF63C296
:103DD000ECFF64C2ECFF65C2ECFF5DC26CF265C231
:103DE00070F264C26FF263C26EF262C26DF20001E1
:103DF00053EC10F0010E0201576FC20E566F5CC2F9
:103E000072F2370E736F0001D5EC16F05BC272F2DE
:103E1000370E0201736F0001D5EC16F0A8EC19F013
:103E200074EF24F0010E02016F6F870E6E6F020EA9
:103E3000706F0001FCEC19F000C05DF2036A020132
:103E40005D514A0FE96E010E0320EA6EEFCF6CF26E
:103E5000010E576FC20E566F5CC272F2370E736F4F
:103E60000001D5EC16F05BC272F2370E0201736FDF
:103E70000001D5EC16F06CC272F2370E0201736FBE
:103E80000001D5EC16F0A8EC19F074EF24F0010E47
:103E900002016F6F870E6E6F020E706F0001FCECF7
:103EA00019F000C05DF2010E02016F6F890E6E6F96
:103EB000020E706F0001FCEC19F000C060F2036AA2
:103EC00002015D514A0FE96E010E0320EA6E60C2E5
:103ED000EFFF5DC2B1F260C2B2F20001C3EC11F0BB
:103EE000010E0201576FC20E566F5CC272F2370E9E
:103EF000736F0001D5EC16F05BC272F2370E02014F
:103F0000736F0001D5EC16F0A8EC19F074EF24F0F3
:103F1000010E02016F6F870E6E6F020E706F00014F
:103F2000FCEC19F000C05DF2036A02015D51320F32
:103F3000E96E010E0320EA6EEFCF6CF2010E576FAF
:103F4000C20E566F5CC272F2370E736F0001D5EC71
:103F500016F05BC272F2370E0201736F0001D5ECEE
:103F600016F06CC272F2370E0201736F0001D5ECCD
:103F700016F0A8EC19F074EF24F0010E02016F6F37
:103F8000870E6E6F020E706F0001FCEC19F000C01E
:103F90005DF2010E02016F6F890E6E6F020E706F7F
:103FA0000001FCEC19F000C05FF2036A02015D51F0
:103FB000320FE96E010E0320EA6E5FC2EFFF186A4E
:103FC000F2BE188EF29E5DC2C9F25FC2CAF2000153
:103FD0005EEC01F018BEF28E010E0201576FC20EA8
:103FE000566F5CC272F2370E736F0001D5EC16F09B
:103FF0005BC272F2370E0201736F0001D5EC16F04E
:10400000A8EC19F074EF24F0010E0201576FC20EF4
:10401000566F5CC272F2370E736F0001D5EC16F06A
:104020005BC272F2370E0201736F0001D5EC16F01D
:104030006FC172F2370E0201736F0001D5EC16F0FA
:104040006EC172F2370E0201736F0001D5EC16F0EB
:10405000A8EC19F074EF24F0010E02016F6F870EC7
:104060006E6F040E706F0001FCEC19F001C06FF16F
:1040700000C06EF15DC26EF26FC170F26EC16FF280
:1040800026EC03F0010E0201576FC20E566F5CC2A0
:1040900072F2370E736F0001D5EC16F05BC272F24C
:1040A000370E0201736F0001D5EC16F0A8EC19F081
:1040B00074EF24F0010E02016F6F870E6E6F020E17
:1040C000706F0001FCEC19F000C05DF2D8900201A5
:1040D0005D35036A6E0FE96E010E0320EA6EECCFC8
:1040E0006DF2ED52EFCF6CF2FF0E6C256E6F7F0E0E
:1040F0006D216F6F010E576FC20E566F5CC272F268
:10410000370E736F0001D5EC16F05BC272F2370EFA
:104110000201736F0001D5EC16F06FC272F2370E18
:104120000201736F0001D5EC16F06EC272F2370E09
:104130000201736F0001D5EC16F0A8EC19F0D4D38E
:10414000010E02016F6F870E6E6F020E706F00011D
:10415000FCEC19F000C05DF2D89002015D35036AF5
:104160006E0F016E010E032201C06CF203C06DF2EE
:10417000010E6F6F890E6E6F040E706F0001FCEC04
:1041800019F06DC2EAFF6CC2E9FF01C0ECFFED520D
:1041900000C0EFFFD89002015D35036A6E0FE96E33
:1041A000010E0320EA6EFF0EEF5C006E7F0EEC58EE
:1041B000036E0050ED52EF6E03C0ECFFD8905D35FA
:1041C000036A6E0FE96E010E0320EA6EECCF6DF20A
:1041D000ED52EFCF6CF25DC26EF26DC270F26CC246
:1041E0006FF2000126EC03F0010E0201576FC20EC0
:1041F000566F5CC272F2370E736F0001D5EC16F089
:104200005BC272F2370E0201736F0001D5EC16F03B
:10421000A8EC19F069D3C282C2B2FED7C4CF67F24C
:104220000201C3CF66F2010E576FC20E566F5CC219
:1042300072F2370E736F0001D5EC16F05BC272F2AA
:10424000370E0201736F0001D5EC16F067C272F2EF
:10425000370E0201736F0001D5EC16F066C272F2E0
:10426000370E0201736F0001D5EC16F0A8EC19F0BF
:104270003BD3010E02016C6F00010DEC14F0010E36
:104280000201576FC20E566F5CC272F2370E736F27
:104290000001D5EC16F05BC272F2370E0201736FAB
:1042A0000001D5EC16F0040E0201686F5D6B5D51E4
:1042B00003083CE35E6B5E51030836E3C20E6825DB
:1042C0006C6F010E6D6FD8B06D2B5D51080DF35002
:1042D0006F6B6E6FD8905E35036A6E25016E6F51FD
:1042E000032201504E0FE96E010E0320EA6EECCF5F
:1042F00071F2ED52EFCF70F26DC257F26CC256F20E
:1043000071C272F2370E736F0001D5EC16F070C2F5
:1043100072F2370E0201736F0001D5EC16F0040E35
:10432000020168275E2BC7D75D2BC1D70001A8EC1F
:1043300019F0DAD2010E02016F6F870E6E6F020E56
:10434000706F0001FCEC19F000C05DF2010E02017B
:104350006F6F890E6E6F020E706F0001FCEC19F02A
:1043600000C05EF202015D51080DF3506D6B6C6F81
:10437000D8905E35036A6C25016E6D5103220150A1
:104380004E0FE96E010E0320EA6EECCF6FF2ED5294
:10439000EFCF6EF2010E576FC20E566F5CC272F213
:1043A000370E736F0001D5EC16F05BC272F2370E58
:1043B0000201736F0001D5EC16F06FC272F2370E76
:1043C0000201736F0001D5EC16F06EC272F2370E67
:1043D0000201736F0001D5EC16F0A8EC19F084D23D
:1043E000010E02016F6F870E6E6F020E706F00017B
:1043F000FCEC19F00101319100B0318131A103D001
:1044000098948F9402D098948F84010E0201576F74
:10441000C20E566F5CC272F2370E736F0001D5EC9C
:1044200016F05BC272F2370E0201736F0001D5EC19
:1044300016F0A8EC19F058D2000E010131B1010EAE
:1044400002016C6F010E576FC20E566F5CC272F2A2
:10445000370E736F0001D5EC16F05BC272F2370EA7
:104460000201736F0001D5EC16F06CC272F2370EC8
:104470000201736F0001D5EC16F0A8EC19F034D2EC
:10448000010E02016F6F870E6E6F020E706F0001DA
:10449000FCEC19F000C05DF202015D51030801E27D
:1044A0005D6B010E6F6F890E6E6F020E706F0001F3
:1044B000FCEC19F000C069F202015D51080DF350E7
:1044C0006D6B6C6F190E6C25E96E000E6D21EA6E36
:1044D00069C2EFFF695302E1010E696F5D51080D7A
:1044E000F3506D6B6C6F190E6C25E96E000E6D212B
:1044F000EA6E69C2EFFF010E6F6F8B0E6E6F020ED8
:10450000706F0001FCEC19F000C06AF202016A5100
:10451000800802E2800E6A6F5D51080DF3506D6BEA
:104520006C6F010E6C25016E000E6D21036E015043
:10453000190FE96E000E0320EA6E6AC2EFFF5D51AB
:10454000080DF3506D6B6C6F060E6C25016E000E3E
:104550006D21036E0150190FE96E000E0320EA6E03
:10456000036A69C270F203C071F2010E736F400EEC
:10457000726F03C075F269C274F200017BEF1BF029
:104580000150010FEF6E000E0220EC6E010E0201D1
:10459000576FC20E566F5CC272F2370E736F000116
:1045A000D5EC16F05BC272F2370E0201736F000198
:1045B000D5EC16F069C272F2370E0201736F00017A
:1045C000D5EC16F06AC272F2370E0201736F000169
:1045D000D5EC16F0A8EC19F087D1010E02016F6F2F
:1045E000870E6E6F020E706F0001FCEC19F000C0B8
:1045F0005DF2010E02016F6F890E6E6F020E706F19
:104600000001FCEC19F000C06BF202015D51080DD5
:10461000F3506D6B6C6F020E6C25016E000E6D21F8
:10462000036E0150190FE96E000E0320EA6E6BC293
:10463000EFFF5D51080DF3506D6B6C6F040E6C2530
:10464000016E000E6D21036E0150190FE96E000E10
:104650000320EA6EEC6AED52EF6A010E576FC20E4C
:10466000566F5CC272F2370E736F0001D5EC16F014
:104670005BC272F2370E0201736F0001D5EC16F0C7
:104680006BC272F2370E0201736F0001D5EC16F0A7
:10469000A8EC19F029D1010E02016F6F870E6E6F21
:1046A000020E706F0001FCEC19F000C05DF2020117
:1046B0005D51080DF3506D6B6C6F020E6C25016E31
:1046C000000E6D21036E0150190FE96E000E0320DC
:1046D000EA6EEFCF6BF2010E576FC20E566F5CC2DF
:1046E00072F2370E736F0001D5EC16F05BC272F2F6
:1046F000370E0201736F0001D5EC16F06BC272F237
:10470000370E0201736F0001D5EC16F0A8EC19F01A
:10471000EBD0010E02016F6F870E6E6F020E706F8D
:104720000001FCEC19F000C05DF202015D51080DC2
:10473000F3506D6B6C6F190E6C25E96E000E6D21D8
:10474000EA6EEFCF6EF25D51080DF350706B6F6F34
:10475000010E6F25016E000E7021036E0150190FBE
:10476000E96E000E0320EA6EEFCF71F2010E576F73
:10477000C20E566F5CC272F2370E736F0001D5EC39
:1047800016F05BC272F2370E0201736F0001D5ECB6
:1047900016F06EC272F2370E0201736F0001D5EC93
:1047A00016F071C272F2370E0201736F0001D5EC80
:1047B00016F0A8EC19F098D0010E02016F6F870E69
:1047C0006E6F020E706F0001FCEC19F000C07EF1FC
:1047D00001017E5304E0949C8B8C036A02D0949C6C
:1047E0008B9C010E0201576FC20E566F5CC272F2B3
:1047F000370E736F0001D5EC16F05BC272F2370E04
:104800000201736F0001D5EC16F0A8EC19F06CD022
:10481000010E0201576FC20E566F5CC272F2370E64
:10482000736F0001D5EC16F05BC272F2370E020115
:10483000736F0001D5EC16F07EC172F2370E0201E3
:10484000736F0001D5EC16F0A8EC19F04DD0010EF5
:104850000201576FC20E566F5CC272F2370E736F51
:104860000001D5EC16F05BC272F2370E0201736FD5
:104870000001D5EC16F07CC172F2370E0201736FA5
:104880000001D5EC16F0A8EC19F02ED0010E0201B3
:104890006F6F870E6E6F020E706F0001FCEC19F0E7
:1048A00000C07FF1010E0201576FC20E566F5CC24D
:1048B00072F2370E736F0001D5EC16F05BC272F224
:1048C000370E0201736F0001D5EC16F0A8EC19F059
:1048D0000BD002016D6B010E6C6F6E6B0001F8EC7A
:1048E00016F0A8EC19F000D008EC12F09298899814
:1048F0002FEF25F002015F6B5E6B5D6B5E515C5DBF
:104900001EE303E15B515D5D1AE2C20E5D25E96EB7
:10491000010E5E21EA6EEFCF62F262C270F2000118
:1049200067EC19F0C20E02015D25E96E010E5E21F1
:10493000EA6EEF505F275D2BD8B45E2BDFD75F1F89
:104940005F39006E0F0E00160050300F606F5F5120
:104950000F0B300F616F6051390802E2070E6027BC
:104960006151390802E2070E612760C270F200014E
:1049700067EC19F061C270F267EC19F0030E0201E6
:10498000706F000167EC19F0000C020164516603BE
:10499000F3CF01F0F4CF00F06703F3500026655128
:1049A0006603F3500020026E000163EF26F0F86A00
:1049B000D09E0D8EFE0E006E0F0E016E020EE96E81
:1049C000000EEA6EEE6A002EFDD7012EFBD7EA6AD2
:1049D000E96AC150C00B0F09C16E070EB46E080E14
:1049E0000101786F796B010E7F6F806B816B020123
:1049F000566B576B000169EF15F0948E01017C6BCB
:104A000082BE7C2B7F531FE07D517C5D1CE0320E0B
:104A10000201B16F00012DEC02F0948E01017C6B5C
:104A200082BE7C2B7D517C5D0EE002016D6B800EA1
:104A30006C6F7CC16EF20001F8EC16F0A8EC19F076
:104A40007CC17DF10101988286B204D00001BCEFE7
:104A50001AF0010131A504D000019FEF1BF0010104
:104A60002B3D06D02C5304E12D5302E12E5353E08D
:104A70002B2D25D02C5323E12D5321E12E531FE163
:104A800002016D6B0B0E6C6F6E6B0001F8EC16F093
:104A9000A8EC19F0010EEA6EC20EE96EE26A390E58
:104AA000E16E780E016EE6CFEEFF012EFCD702011B
:104AB0005C6B780E5B6F00011DDF27D001012B516D
:104AC000020824E12C5322E12D5320E12E531EE154
:104AD00002016D6B0B0E6C6F6E6B0001F8EC16F043
:104AE000A8EC19F0010EEA6EC20EE96EE26AB10E90
:104AF000E16E780E016EE6CFEEFF012EFCD70201CB
:104B00005C6B780E5B6F0001F5DE01012E6B2D6B87
:104B10002C6BFF0E2B6F02015A6B5A510308D8A061
:104B2000E1D05A51080DF3505C6B5B6F020E5B25B0
:104B3000016E000E5C21036E0150190FE96E000E2C
:104B40000320EA6EEF2CCCD05A51080DF3505C6B69
:104B50005B6F040E5B25016E000E5C21036E01503D
:104B6000190FE96E000E0320EA6EECCF5EF2ED52F3
:104B7000EFCF5DF25A51080DF350606B5F6F060E78
:104B80005F25016E000E6021036E0150190FE96E62
:104B9000000E0320EA6EECCF03F0ED52EFCF01F0F0
:104BA00003505E5DD8A09CD004E101505D5DD8A0AB
:104BB00097D05A51080DF3505C6B5B6F040E5B2568
:104BC000016E000E5C21036E0150190FE96E000E9C
:104BD0000320EA6EEC6AED52EF6A5A51080DF35069
:104BE0005C6B5B6F030E5B25016E000E5C21036E38
:104BF0000150190FE96E000E0320EA6EEF2A5A5198
:104C0000080DF3505C6B5B6F030E5B25016E000EAD
:104C10005C21036E0150190FE96E000E0320EA6E4D
:104C2000EF501F0812E25A51080DF3505C6B5B6F96
:104C3000030E5B25016E000E5C21036E0150190FFF
:104C4000E96E000E0320EA6EEF6A5A51080DF35028
:104C50005C6B5B6F010E5B25016E000E5C21036EC9
:104C60000150190FE96E000E0320EA6EEFCF5DF2DE
:104C70005A51080DF3505F6B5E6F030E5E25016E97
:104C8000000E5F21036E0150190FE96E000E032024
:104C9000EA6ED890EF34036AF2CF61F2F29E00011F
:104CA00055EC00F00900F5CF03F0020161BFF28E70
:104CB000626F03C063F2656B5DC264F203C067F2AA
:104CC000666F000162D602C064F201C063F25AC28C
:104CD0006EF202C070F201C06FF226EC03F0020126
:104CE0005A2B1BD7938081B008D0640EB16F00019E
:104CF0002DEC02F0938081B000D000017ED603003D
:020000040030CA
:0E00000000260C1E838381000FC00FE00F400E
:00000001FF
